:100000000C9495020C94D9020C94D9020C94D90248
:100010000C94D9020C94D9020C94D9020C94D902F4
:100020000C94D9020C94D9020C94670E0C94390FDD
:100030000C94D9020C94D9020C94D9020C94D902D4
:100040000C94D9020C94A3220C94D9020C94D902DA
:100050000C94D9020C94851D0C94D9020C94D902ED
:100060000C94D9020C94D9020C94D9020C94D902A4
:100070000C94D9020C94D9020C94D9020C94D90294
:100080000C94D9020C94D9020C94D9020C94D90284
:100090000C94D9020C94D9020C94D9020C94D90274
:1000A0000C94D9020C94D9020C94D902A60FC80F53
:1000B000B610C80FB6100D103010B610851098107D
:1000C0006913691395139513D813F8135315531522
:1000D00003145315B014B0144415531553154D158E
:1000E000BD14BD14BD14BD14BD14BD14BD14BD1488
:1000F000BD14BD14BD14BD14BD14BD14BD14BD1478
:10010000CE14DB14E214E914F314021902E3000123
:10011000E3011900020602E30001E30106000213F5
:100120000001E00104020402E001130002290001C1
:10013000E00104020402E00129000000F4A2002210
:1001400030A135002B003161C200C10000001E004B
:10015000140004001D0001534D001F001A0016007A
:100160001B00E0004C002000080007000600E20031
:100170002A002100150009001900E3004A002200AE
:1001800017000A00050000000A3029006B67000014
:100190006D6F00000B3066006C6700006E6F000032
:1001A0000C3023001C000B00110000000D30240057
:1001B00018000D001000E7004B0025000C000E0099
:1001C0003600E6002C00260012000F0037002F61D9
:1001D00028002700130033003800C3004E002D0014
:1001E0002E003461C200C10000000000FF00FE00CC
:1001F000FD00000000000000000000000000010001
:100200000000F400F900F200FB0000000000F5001F
:10021000F000F100000000000000F600FA00F3001A
:10022000FC000000000000000000000000000000D2
:1002300000000000000000000000000000002B0291
:100240002B0000005800000000009C005F005C00D4
:10025000590000000000540060005D005A00620078
:100260000000550061005E005B0063000000230297
:100270005700560067008500010026022702000093
:10028000000001000000000000000000000000006D
:100290000000000000003900E100010000003A0009
:1002A000AD00B0000000000000003B00BC00AC004E
:1002B0000000010000003C00AF00AE0000000100A3
:1002C00000003D00BB00AB000000010000003E004C
:1002D000000000000000000000003F0001000000DE
:1002E00001000000000040000100000001000000CB
:1002F000000041000000500000000000000042002B
:100300000000510000000100000043000000520006
:10031000000001000000440000004F000000010048
:100320000000450000000000000000000000A900DF
:10033000AA00A800E50001000000160345007200B5
:1003400067006F0044006F007800200045005A00ED
:10035000000016034500720067006F0044006F0044
:100360007800200045005A00000004030904090237
:100370006D00040100A0FA0904000001030101005E
:100380000921110100012240000705810308000A2C
:1003900009040100010301020009211101000122E9
:1003A0004D000705820308000A090402000103004A
:1003B000000009211101000122360007058303080E
:1003C000000A0904030001030000000921110100D3
:1003D00001223900070584031000011201100100F9
:1003E000000008EDFE0713010001020001050109EC
:1003F00006A101050719E029E715002501950875F3
:1004000001810205081901290595057501910295DB
:10041000017503910105071900297715002501953C
:100420007875018102C005010980A10185021601CC
:100430000026B7001A01002AB70075109501810047
:10044000C0050C0901A1018503160100269C021AB2
:1004500001002A9C02751095018100C00501090266
:10046000A1010901A10005091901290515002501AE
:10047000950575018102950175038101050109301A
:1004800009311581257F9502750881060938158186
:10049000257F950175088106050C0A38021581250E
:1004A0007F950175088106C0C005010906A10105F7
:1004B0000719E029E71500250195087501810295C6
:1004C0000175088101050819012905950575019136
:1004D000029501750391010507190029FF150026F2
:1004E000FF00950675088100C000000000000000B4
:1004F00000000000010204060A0F17202C3A4A5D92
:1005000071879DB3C7DAE9F5FCFFFCF5E9DAC7B3FB
:100510009D87715D4A3A2C20170F0A0604020100DC
:100520000000000000000000000011241FBECFEFFB
:10053000DAE0DEBFCDBF04B603FE24C08091030223
:1005400090910402A0910502B09106028730904B71
:10055000A740B04BB9F4109203021092040210921B
:1005600005021092060214BE84B7877F84BF88E11B
:100570000FB6F89480936000109260000FBEE0E028
:10058000FFE3099511E0A0E0B1E0E4EDF8E402C07A
:1005900005900D92A433B107D9F712E0A4E3B1E0BE
:1005A00001C01D92A330B107E1F70E94AF0B0C947C
:1005B00068240C9400001092B9008AE08093B8007F
:1005C000089594EA9093BC009091BC0097FFFCCFF3
:1005D0009091B900987F983021F0903111F081E02E
:1005E00008958093BB0084E88093BC008091BC0098
:1005F00087FFFCCF8091B900887F883111F080346B
:1006000071F780E0089584E98093BC008091BC007C
:1006100084FDFCCF08958093BB0084E88093BC00E8
:100620008091BC0087FFFCCF9091B900987F81E05A
:10063000983209F480E0089584E88093BC008091AA
:10064000BC0087FFFCCF8091BB00089580B38C7005
:1006500080BB81B3836F81BB0895809101018111BB
:1006600015C080E40E94E1028093010181110CC059
:1006700082E10E940B0380930101811105C08FEF7D
:100680000E940B03809301010E94030384B1807FC9
:1006900084B985B1807F85B98AB1837F8AB98BB1EE
:1006A000837F8BB93E98469808950E94F704809303
:1006B00001010E942D030E942603A5E3B1E0E3E4BB
:1006C000F1E08EE08E0F11921D928E13FCCF0C94F0
:1006D000E1040E94F704809301010E942D030E940F
:1006E0002603A5E3B1E0E3E4F1E08EE08E0F119282
:1006F0001D928E13FCCF0895BF92CF92DF92EF929E
:10070000FF920F931F93CF93DF9380910101882372
:1007100079F0809134018F5F80933401811108C09A
:100720000E94F70480930101811102C00E94890494
:1007300005E311E0C0E0D0E0DD24D39482E0C82ED0
:10074000EE24E394F12CC730D10500F5809101012E
:10075000811164C080E40E94E10280930101811153
:1007600012C082E10E940B038093010181110BC032
:10077000C7010C2E01C0880F0A94EAF780950E94E9
:100780000B03809301010E94030348C0CA30A1F00B
:1007900028F4C83059F0C93061F005C0CC3089F078
:1007A00070F0CD3089F0209A289810C0219A2998AD
:1007B0000DC0229A2A980AC0239A2B9807C0529AF1
:1007C00001C0539A5B9802C03E9A469890EA9A9567
:1007D000F1F79FB1799902C082E001C080E0917089
:1007E0009D25982B7C9902C084E001C080E0892B74
:1007F0007D9902C038E001C030E0832B7E9902C0B1
:1008000020E101C020E0822B9FB19095991F99278C
:10081000991F9295990F907E892B0FC080910101AD
:10082000811149C080E40E94E10280930101882384
:1008300079F1B12C0E9403038B2DF8019081981758
:1008400019F08083C09200010E942D0321960F5F52
:100850001F4FCE30D10509F076CF8091000188235B
:1008600061F1815080930001882339F08FE99FE086
:100870000197F1F700C0000020C0A3E4B1E0E5E378
:10088000F1E0CF01825F91919D938E13FCCF15C053
:1008900083E10E940B03809301018111CACF81E49F
:1008A0000E94E102809301018111C3CF0E941C03C9
:1008B000B82EB094BFCF80E0C0CF0E94870481E003
:1008C000DF91CF911F910F91FF90EF90DF90CF902C
:1008D000BF900895E82FF0E0ED5BFE4F8081089512
:1008E00008950F931F93CF93DF93C3E4D1E010E0FB
:1008F0000C2F025F899190E00E94AC1C180F0C1322
:10090000F9CF812FDF91CF911F910F9108950C9412
:100910007A0556985E9825982D9826982E982798AF
:100920002F988FEF90E090938900809388009093A8
:100930008B0080938A0090938D0080938C00259A81
:100940002D9A2FEF80E792E0215080409040E1F710
:1009500000C00000269A2E9A2FEF80E792E02150E7
:1009600080409040E1F700C00000279A2F9A2FEFB7
:1009700080E792E0215080409040E1F700C0000005
:1009800025982D982FEF80E792E0215080409040ED
:10099000E1F700C0000026982E982FEF80E792E044
:1009A000215080409040E1F700C0000027982F9828
:1009B00056985E9825982D9826982E9827982F98C7
:1009C000089589EA8093800089E0809381002498CB
:1009D0002C983F988AB18F748AB96E98479A8BB1D8
:1009E000806B8BB9769A0E9489040C94790580E219
:1009F000809301018091510181110EC00E94DB02A0
:100A000081E0809351012FEF83ED90E321508040EE
:100A10009040E1F700C0000080E40E94E102809372
:100A2000010181112EC00E940B03809301018111ED
:100A300028C00E940B0380930101811122C08FE323
:100A40000E940B038093010181111BC00E940303CC
:100A500080E40E94E10280930101811112C08CE0C8
:100A60000E940B038093010181110BC00E940B03B4
:100A700080930101811105C08FE30E940B038093D5
:100A800001010E940303809101010895FC016B3074
:100A900079F018F46A3031F01DC06C3079F06D30A7
:100AA00099F018C08281811118C08CE291E00895FC
:100AB0008281811115C08EE191E0089582818111BA
:100AC00012C084E191E00895828181110FC08AE013
:100AD00091E0089580E090E008958FE291E008951C
:100AE00081E291E0089589E191E008958FE091E03D
:100AF00008950895CF936091BF017091C0018091D6
:100B0000C1019091C2010E94B81CC82F56985E98EE
:100B100025982D9826982E9827982F988FE090E06A
:100B2000909389008093880090938B0080938A0033
:100B300090938D0080938C00CC2329F0C13029F450
:100B4000C093520102C01092520180915201813033
:100B500011F4279A2F9A0E94EF10867011F0259AAF
:100B60002D9AC23041F40E94351B811104C0279890
:100B70002F98269A2E9AE0910E01F0910F01808114
:100B8000982F927259F08D7D49F48FEF90E09093F9
:100B9000890080938800259A2D9A08C00E94621CC3
:100BA000827221F00E94081B882379F3CF91089567
:100BB00081E0089581E008950C94DA050895282FC6
:100BC000882339F090E02A3010F44D960895069766
:100BD000089587E290E00895AF92BF92DF92EF927E
:100BE000FF920F931F93CF93DF938C01FC01C08181
:100BF000D181CE010E94B11ABE010E945C09EC01B4
:100C0000B8010E94DC05882309F4C9C1F80182817A
:100C1000882309F4BEC080915F0181111FC0C431D7
:100C2000F0E7DF0709F0B5C10E94DE0581E080939F
:100C30005F010E944F1D90935E0180935D011092B1
:100C40005601109258011092570110925A011092B9
:100C5000590110925C0110925B01A1C180915D016C
:100C600090915E010E945B1D883C910570F480911B
:100C70005601E82FF0E0EE0FFF1FE95AFE4FD18337
:100C8000C0838F5F809356018AC1C13020E8D207AC
:100C900008F451C0F8018281882309F47EC05E0106
:100CA000E894B7F880915501813079F050F08230A6
:100CB000C1F482EE0E940B1287E50E940B1287E5B9
:100CC0000EC082EE0E940B120CC080EE0E940B122E
:100CD00081EE0E940B1288E10E940B1288E10E94B3
:100CE000D3128CE0E82EF12CC5010E2C02C0969593
:100CF00087950A94E2F78F700E94DF05D82E0E9434
:100D00000B128D2D0E94D312F4E0EF1AF1082CEF94
:100D1000E2162FEFF20641F780915501813029F05C
:100D200010F0823041F482EE04C080EE0E94D312B3
:100D300081EE0E94D312C43180E7D80768F4C23034
:100D400090E7D90708F046C0C115E0E7DE0771F06B
:100D5000C130D047A1F10CC1C33320E7D20709F459
:100D6000D8C0C433D04709F4EBC002C1F801828176
:100D7000882309F402C10E94B815FFEF24E38CE038
:100D8000F15020408040E1F700C000000E94AA1D01
:100D900006C1C13080E8D80770F2C43120E7D2071D
:100DA00008F0B3C0C23080E7D807A0F4C11590E7BF
:100DB000D90709F4E2C0C130D04709F0D9C0F80121
:100DC0008281882309F4D9C08091E10181608093F8
:100DD000E101E5C0F8018281882309F4CEC00E94B8
:100DE000041E811102C00E94EA1D0E94171E90E09D
:100DF0009093F5018093F401C230F0E7DF0721F40E
:100E00008091F40181607AC0C33020E7D20721F4D9
:100E10008091F401826072C0C43080E7D80721F469
:100E20008091F40184606AC0C53090E7D90719F455
:100E30008091F40127C0C630E0E7DE0721F48091FD
:100E4000F40180615BC0C730F0E7DF0721F48091D7
:100E5000F401806253C0C83020E7D20721F48091AA
:100E6000F40180644BC0C93080E7D80721F4809139
:100E7000F401806843C0CA3090E7D90729F4809113
:100E8000F401846088603AC0CB30E0E7DE0721F4EB
:100E90008091F4018E7F32C0CC30F0E7DF0721F47F
:100EA0008091F4018D7F2AC0CD3020E7D20721F454
:100EB0008091F4018B7F22C0CE3080E7D80719F4EF
:100EC0008091F4011AC08091F401CF3090E7D907E6
:100ED00011F48F7E13C0C031E0E7DE0711F48F7D7F
:100EE0000DC0C131F0E7DF0711F48F7B07C0C231BD
:100EF000D04711F48F7702C08B7F877F8093F401F6
:100F00008091F4010E941B1E4AC0C333F0E7DF0743
:100F1000A1F4F8018281882321F01092530182E02C
:100F200016C080915301811106C086E20E940B1207
:100F300086E20E94D31282E018C0C433D047C1F4C5
:100F4000F8018281882331F01092540180E20E94DE
:100F5000221325C080915401811106C087E20E94AE
:100F60000B1287E20E94D31280E20E94291317C05D
:100F700081E08093530180935401C801DF91CF91A8
:100F80001F910F91FF90EF90DF90BF90AF900C9466
:100F9000D805C130F0E8DF0708F081CECCCE80E084
:100FA000DF91CF911F910F91FF90EF90DF90BF9055
:100FB000AF90089526E0729FF001112444E5849FCC
:100FC000E00DF11D1124E60FF11DEE0FFF1FEE5B8A
:100FD000FE4F859194910E946E09811560E49607F9
:100FE000B0F5811570E3970708F0DEC0803E9105EB
:100FF000D8F4803C910508F06CC0883A910578F4EB
:10100000853A910508F06BC08130910509F452C111
:1010100008F40FC18430910508F04CC10AC18B3B24
:10102000910508F467C005C18F3F910509F048F4A8
:10103000803F910508F0ADC0883E910508F43AC1A3
:10104000F8C0811520E2920708F0A5C00895811527
:1010500043E5940790F4811562E5960708F0C8C04F
:10106000811571E5970708F0BEC0811520E592074C
:1010700008F09DC09F70906A0895811545E594071A
:10108000D8F4811564E5960708F0C8C0482F469546
:10109000469570E2479FA00111248370992721E0B3
:1010A00030E0B90102C0660F771F8A95E2F7CB01E5
:1010B000842B952B9A680895811576E5970708F497
:1010C000B2C09C0130562115304108F0B2C09F706B
:1010D000AEC0FC01EE0FFF1FE654F04062C0853A3F
:1010E000910509F4A9C0863A910509F0A8C082E8E3
:1010F00090E40895883A910509F4A4C0893A9105CD
:1011000009F4A3C08A3A910509F4A2C08B3A91056B
:1011100009F4A1C08C3A910509F4A0C08D3A91055B
:1011200009F49FC0803B910509F49EC08E3A910559
:1011300009F49DC08F3A910509F49CC0813B91054B
:1011400009F49BC0823B910509F49AC0833B910549
:1011500009F499C0843B910509F498C0853B910539
:1011600009F497C0863B910509F496C0873B910529
:1011700009F495C0883B910509F494C0893B910519
:1011800009F493C08A3B910509F492C080E094E48D
:10119000089590650895FC01FF70EE0FFF1FE65C57
:1011A000FE4F8591949108959927906C0895482F4A
:1011B000437021E030E002C0220F331F4A95E2F76E
:1011C0003C68AC0164E0569547956A95E1F7437039
:1011D000342B8F708695869560E2869FC00111241E
:1011E000822B932B0895982F8827816F906A0895FA
:1011F000482F4695469570E2479FA00111248370C1
:10120000992721E030E0B90102C0660F771F8A9567
:10121000E2F7CB01842B952B9C680895982F8827A3
:10122000846F906A08958F719927982F882790620C
:10123000089580E090E0089581E890E4089583E8BF
:1012400090E4089582EE94E4089589EE94E408957C
:101250008AEE94E4089585EB94E4089586EB94E493
:10126000089587EB94E408958CEC94E408958DEC54
:1012700094E4089583E895E408958AE895E4089550
:1012800082E995E4089584E995E4089581E296E47D
:10129000089583E296E4089584E296E4089585E251
:1012A00096E4089586E296E4089587E296E4089528
:1012B0008AE296E40895089596E0799FF00111245A
:1012C00094E5899FE00DF11D1124E60FF11DEE0F4D
:1012D000FF1FEE5BFE4F8591949108958238910532
:1012E00049F1B0F48133910509F458C048F48932CA
:1012F000910509F44EC08A32910509F454C008954D
:101300008533910509F440C08933910599F008951A
:10131000833E910529F138F4803E910591F0823E9B
:101320009105A1F00895863E9105F9F0873E91055B
:1013300031F108952091F40120FD3AC021FD38C01B
:1013400008958091F40180FD35C032C08091F40190
:1013500082FF32C08091F40184FD30C083EE39C039
:101360008091F40182FD28C0F5CF8091F40183FFC4
:1013700027C08091F40184FD21C087EE2AC08091AE
:10138000F40183FD1DC0F5CF8091F40185FD1AC0E5
:101390001BC08091F40185FD17C014C08091F40139
:1013A00086FD14C015C08091F40186FD11C00EC0E9
:1013B00080EE0FC089E30DC082EE0BC080E009C053
:1013C00086EE07C089E205C085E303C08AE201C05A
:1013D00081E390E0089508950C94EB0980917001E9
:1013E0000895CF93DF9300D01F92CDB7DEB79C0155
:1013F0008091FA01843019F593E099833B832A8325
:101400009093E9008FEF9091E800815095FD06C020
:1014100095ED9A95F1F700008111F5CF8091E800E4
:1014200085FF0DC040E050E063E070E0CE01019622
:101430000E94570C8091E8008E778093E8000F900F
:101440000F900F90DF91CF910895CF93DF9300D04D
:101450001F92CDB7DEB72091FA01243021F522E0AA
:1014600029839B838A8383E08093E9008FEF9091A7
:10147000E800815095FD06C095ED9A95F1F70000C2
:101480008111F5CF8091E80085FF0DC040E050E06C
:1014900063E070E0CE0101960E94570C8091E80055
:1014A0008E778093E8000F900F900F90DF91CF918F
:1014B00008952091FA012430F1F422E02093E9000C
:1014C0002FEF3091E800215035FD06C035ED3A95FB
:1014D000F1F700002111F5CF2091E80025FF0BC0A6
:1014E00040E050E065E070E00E94570C8091E80019
:1014F0008E778093E8000895CF93DF93EC0190916D
:10150000FA01943009F046C080910C018823D9F08B
:1015100080910D018823B9F09093E9008FEF9091AD
:10152000E800815095FD06C095E19A95F1F700001D
:101530008111F5CF8091E80085FF2CC040E050E09C
:1015400060E170E017C081E08093E9008FEF909137
:10155000E800815095FD06C095ED9A95F1F70000E1
:101560008111F5CF8091E80085FF14C040E050E084
:1015700068E070E0CE010E94570C8091E8008E7701
:101580008093E80080E1FE01A0E6B1E001900D92B9
:101590008A95E1F7DF91CF9108958091F90181114A
:1015A00009C00E94EC0D0E94490E8091E200846007
:1015B0008093E20008951092F901089508950C9423
:1015C00090220E94401D0E9496220E94EF100C94CF
:1015D000EC0942E061EC81E00E94660D42E061ECC2
:1015E00082E00E94660D42E061EC83E00E94660D9D
:1015F00042E161EC84E00C94660D8091FC01833043
:1016000009F455C030F4813071F0823009F48EC095
:1016100008958A3009F47AC08B3009F460C08930AB
:1016200009F09CC020C08091FB01813A09F096C06E
:101630008091E800877F8093E8008091FF0190917E
:101640000002892B21F460E180E691E003C060E0B4
:1016500080E090E070E00E94A20C8091E8008B771F
:101660008093E80008958091FB01813209F076C0F3
:101670008091FF0190910002009719F0039709F003
:101680006DC08091E800877F8093E8008091E8003A
:1016900082FD05C08091FA018111F8CF5FC0809171
:1016A000F100809370018091E8008B7753C08091A6
:1016B000FB01813A09F052C08091FF019091000234
:1016C000892B09F04BC08091E800877F8093E80068
:1016D0008091E80080FFFCCF80910C0136C08091A2
:1016E000FB018132D9F58091FF0190910002892B95
:1016F000A9F58091E800877F8093E8000E949B0D08
:101700008091FD0180930C010C94B8158091FB0130
:10171000813221F58091E800877F8093E8000E9464
:101720009B0D8091FE018093710108958091FB01D2
:10173000813AA1F48091E800877F8093E80080914E
:10174000E80080FFFCCF809171018093F1008091CF
:10175000E8008E778093E8000C949B0D089584B781
:10176000877F84BF88E10FB6F89480936000109261
:1017700060000FBE80E880936100109261000E94BB
:101780003E110E94EC0D0E94490E8091E20084609F
:101790008093E20078940E94CF100E94401182E072
:1017A00091E00E94EA100E947E228091FA01853029
:1017B00069F40E94081D8091F8018823B1F30E940A
:1017C000321D882391F30E94410CEFCF0E944611F5
:1017D000ECCF292F332723303105C9F064F42130B1
:1017E000310581F02230310509F043C08DE690E0EB
:1017F0002EE633E042C021323105F1F022323105CC
:1018000041F137C082E190E02BED33E036C09927FB
:101810008130910541F08230910541F0892B49F5E5
:10182000EAE6F3E005C0E2E5F3E002C0EAE3F3E054
:10183000849190E09F0121C06430D8F4E62FF0E05D
:10184000EE0FFF1FEE5DFE4F2081318189E090E0B9
:1018500014C0643070F470E0FB01EE0FFF1FE65E11
:10186000FE4F20813181FB01EA5EFE4F808190E0D6
:1018700004C080E090E020E030E0FA013183208372
:10188000089580E189BD82E189BD09B400FEFDCFE4
:101890008091D8008F7D8093D8008091E000826095
:1018A0008093E0008091E00081FDFCCF0895CF920D
:1018B000DF92EF92FF920F931F93CF93DF93EC0190
:1018C0008B016A010E94BA0D811133C0C114D10489
:1018D00039F0F60180819181081B190BC80FD91FBF
:1018E000E12CF12C0115110519F18091E80085FD1D
:1018F00016C08091E8008E778093E800C114D1046F
:1019000049F0F60180819181E80EF91EF182E082B2
:1019100085E00FC00E94BA0D882321F30AC0899187
:101920008093F10001501109FFEFEF1AFF0ADACF9F
:1019300080E0DF91CF911F910F91FF90EF90DF90AA
:10194000CF900895209101023091020226173707A7
:1019500048F06115710539F42091E8002E77209345
:10196000E80001C0B90140E061157105A9F12091BD
:10197000FA01222309F443C0253009F442C0209122
:10198000E80023FD40C02091E80022FD32C02091F4
:10199000E80020FFE9CF4091F3002091F20030E011
:1019A000342BFC01CF016115710559F02830310548
:1019B00040F481918093F100615071092F5F3F4F96
:1019C000F1CF41E02830310509F040E02091E800F6
:1019D0002E772093E800C8CF4111C9CF0AC080916B
:1019E000FA01882361F0853061F08091E80083FD81
:1019F0000AC08091E80082FFF2CF80E0089582E083
:101A0000089583E0089581E00895209101023091C6
:101A100002022617370748F06115710539F4209145
:101A2000E8002E772093E80001C0B901FC0120E016
:101A30006115710591F18091FA01882309F440C084
:101A4000853009F43FC08091E80083FD3DC080915E
:101A5000E80082FD2FC08091E80080FFE9CF20914F
:101A6000F3008091F20090E0922B6115710559F01E
:101A70008830910540F424912093F1003196615013
:101A800071090196F2CF21E0089709F020E08091DA
:101A9000E8008E778093E800CBCF2111CCCF0AC02D
:101AA0008091FA01882361F0853061F08091E8002F
:101AB00083FD0AC08091E80082FFF2CF80E00895A4
:101AC00082E0089583E0089581E00895982F97308B
:101AD00058F59093E900981739F07091EC00209137
:101AE000ED005091F00003C0242F762F50E021FF2D
:101AF00019C03091EB003E7F3093EB003091ED0048
:101B00003D7F3093ED003091EB0031603093EB007E
:101B10007093EC002093ED005093F0002091EE00C4
:101B200027FF07C09F5FD3CF8F708093E90081E0CC
:101B3000089580E008958091FB0187FF11C0809196
:101B4000E80082FD05C08091FA018111F8CF11C033
:101B50008091E8008B770BC08091FA01882349F0CF
:101B60008091E80080FFF8CF8091E8008E77809325
:101B7000E80008952091E4003091E50095E6409159
:101B8000EC00842F817040FF22C08091E80080FD2E
:101B90001CC08091FA01882391F0853091F08091EA
:101BA000EB0085FD10C04091E4005091E500421724
:101BB000530729F39A01915011F784E0089582E0C8
:101BC000089583E0089581E0089580E008954091AC
:101BD000E80042FFDECF08950E945A0E0E94620E76
:101BE000E0EEF0E0808181608083E8EDF0E08081CC
:101BF0008F77808319BCA7EDB0E08C918E7F8C939A
:101C000080818F7E80831092F90108950F931F9336
:101C1000CF93DF930E945A0E0E94620EC8EDD0E06F
:101C200088818F77888388818068888388818F7D89
:101C3000888319BC1092FA011092F6011092F801F3
:101C40001092F70100EE10E0F80180818B7F808315
:101C500088818160888342E060E080E00E94660DB8
:101C6000E1EEF0E080818E7F8083E2EEF0E0808123
:101C700081608083808188608083F80180818E7F8D
:101C80008083888180618883DF91CF911F910F913C
:101C90000895E8EDF0E080818F7E8083E7EDF0E04D
:101CA00080818160808384E082BF81E08093F9013C
:101CB0000C94060EE8EDF0E080818E7F8083109218
:101CC000E20008951092DA001092E10008951F9248
:101CD0000F920FB60F9211242F933F934F935F9360
:101CE0006F937F938F939F93AF93BF93EF93FF93E4
:101CF0008091E10082FF0BC08091E20082FF07C06B
:101D00008091E1008B7F8093E1000E94CE10809152
:101D1000DA0080FF1FC08091D80080FF1BC0809137
:101D2000DA008E7F8093DA008091D90080FF0DC0A9
:101D300080E189BD82E189BD09B400FEFDCF81E06B
:101D40008093FA010E94CD0A05C019BC1092FA01D5
:101D50000E94DB0A8091E10080FF19C08091E200BF
:101D600080FF15C08091E2008E7F8093E200809119
:101D7000E20080618093E2008091D80080628093CD
:101D8000D80019BC85E08093FA010E94DF0A809197
:101D9000E10084FF30C08091E20084FF2CC080E12C
:101DA00089BD82E189BD09B400FEFDCF8091D800D4
:101DB0008F7D8093D8008091E1008F7E8093E10039
:101DC0008091E2008F7E8093E2008091E20081604A
:101DD0008093E2008091F601882311F084E007C02F
:101DE0008091E30087FD02C081E001C083E0809321
:101DF000FA010E94E10A8091E10083FF29C08091ED
:101E0000E20083FF25C08091E100877F8093E1009D
:101E100082E08093FA011092F6018091E1008E7FBA
:101E20008093E1008091E2008E7F8093E2008091B8
:101E3000E20080618093E20042E060E080E00E9486
:101E4000660D8091F00088608093F0000E94DE0AA9
:101E5000FF91EF91BF91AF919F918F917F916F9182
:101E60005F914F913F912F910F900FBE0F901F9058
:101E700018951F920F920FB60F9211242F933F9334
:101E80004F935F936F937F938F939F93AF93BF9382
:101E9000CF93DF93EF93FF93C091E900CF708091D0
:101EA000EC00D82FD17080FDD0E81092E90080912D
:101EB000F000877F8093F00078940E947D0F10924D
:101EC000E9008091F00088608093F000CD2BCF7006
:101ED000C093E900FF91EF91DF91CF91BF91AF9156
:101EE0009F918F917F916F915F914F913F912F9132
:101EF0000F900FBE0F901F9018951F93CF93DF93F5
:101F0000CDB7DEB7AA970FB6F894DEBF0FBECDBF30
:101F1000EBEFF1E088E08E0F9091F10091938E133A
:101F2000FBCF0E94FD0A8091E80083FF1FC18091D2
:101F3000FB019091FC01492F50E04A30510508F017
:101F400015C1FA01EA5AFF4F0C941824803881F029
:101F5000823809F00BC18091FF018F708093E900F6
:101F60008091EB0085FB882780F91092E90006C07C
:101F70008091F7019091F801911182609091E800B1
:101F8000977F9093E8008093F1001092F100C8C011
:101F9000282F2D7F09F0EAC0882319F0823061F0E4
:101FA000E5C08091FD01813009F0E0C0933009F077
:101FB00080E08093F8012BC08091FD01811127C042
:101FC0008091FF018F7009F4D1C08093E9002091C6
:101FD000EB0020FF1CC0933021F48091EB00806265
:101FE00014C09091EB0090619093EB0021E030E001
:101FF000A90102C0440F551F8A95E2F74093EA00F9
:102000001092EA008091EB0088608093EB001092C0
:10201000E9008091E800877F86C08111A7C01091F8
:10202000FD011F778091E3008078812B8093E3008E
:102030008091E800877F8093E8000E949B0D80914B
:10204000E80080FFFCCF8091E30080688093E3008C
:10205000111102C082E001C083E08093FA0186C0C2
:102060008058823008F082C08091FD019091FE017D
:102070008C3D53E0950779F583E08A838AE2898372
:102080004FB7F894DE01139620E03EE051E2E32FD3
:10209000F0E050935700E49120FF03C0E295EF7009
:1020A0003F5FEF708E2F90E0EA3010F0C79601C0CE
:1020B000C0968D939D932F5F243149F74FBF809138
:1020C000E800877F8093E8006AE270E0CE01019625
:1020D0000E94A20C14C0AE014F5F5F4F6091FF01E0
:1020E0000E94E90BBC01009709F440C09091E80000
:1020F000977F9093E80089819A810E94050D8091D5
:10210000E8008B778093E80031C0803879F58091C2
:10211000E800877F8093E8008091F6018093F100CA
:102120008091E8008E778093E8000E949B0D1EC08E
:1021300081111CC09091FD019230C0F48091E800A3
:10214000877F8093E8009093F6010E949B0D809119
:10215000F601811106C08091E30087FD02C081E095
:1021600001C084E08093FA010E94E90A8091E800AE
:1021700083FF0AC08091E800877F8093E800809108
:10218000EB0080628093EB00AA960FB6F894DEBF56
:102190000FBECDBFDF91CF911F9108950895CF93CA
:1021A0008091FA018823A1F0C091E900CF7090914D
:1021B000EC00892F817090FD80E8C82B1092E90017
:1021C0008091E80083FD0E947D0FCF70C093E900ED
:1021D000CF91089590937701809376010895E091CF
:1021E0007601F0917701309721F00190F081E02D98
:1021F000099480E00895E0917601F091770130979D
:1022000021F00280F381E02D09940895E091760198
:10221000F0917701309721F00480F581E02D099449
:10222000089520917401309175018217930771F020
:102230009093750180937401E0917601F09177019C
:10224000309721F00680F781E02D099408952091C0
:102250007201309173018217930771F090937301AB
:1022600080937201E0917601F0917701309721F02F
:102270000084F185E02D0994089508950C943D1192
:102280000E94461D0E9455030C94CC1D9F92AF9254
:10229000BF92CF92DF92EF92FF920F931F93CF9353
:1022A000DF9300D000D000D0CDB7DEB70E947C0312
:1022B0000DE010E0AA24A394B12C902E802F0E9450
:1022C0006A04980127583E4F6901F901F080F82609
:1022D000A1F40150110988F78FEF89838A831B824B
:1022E0000E944F1D8160782F9D838C8349815A8184
:1022F0006B818D810E94DD112FC09091E10191FFD2
:1023000004C08E830E9470048E8125E030E0A50118
:10231000022E01C0440F0A94EAF7E42E4F21C1F0C7
:1023200029839A828E2191E009F490E09B830E9498
:102330004F1D8160782F9D838C8349815A816B81E9
:102340008D810E94DD11F6018081E826E08204C0C3
:1023500021503109E0F6BDCF0E949A1F10917801FB
:102360000E94EF101817B9F00E94EF1080937801C7
:1023700026960FB6F894DEBF0FBECDBFDF91CF918A
:102380001F910F91FF90EF90DF90CF90BF90AF9093
:102390009F900C94EC0926960FB6F894DEBF0FBE02
:1023A000CDBFDF91CF911F910F91FF90EF90DF9004
:1023B000CF90BF90AF909F900895CF93DF93CDB70C
:1023C000DEB72B970FB6F894DEBF0FBECDBF4F839D
:1023D000588769877A878B87DE01119686E0FD0131
:1023E00011928A95E9F785E0FE01379601900D92EA
:1023F0008A95E1F749815A816B817C818D819E812B
:102400000E9456182B960FB6F894DEBF0FBECDBFB4
:10241000DF91CF910895CF93882309F4C2C0C82FCC
:10242000823859F40E94EF1081FDBBC089E30E94FD
:10243000991B0E94761C89E30CC0833879F40E94B2
:10244000EF1080FDAEC083E50E94991B0E94761CB0
:1024500083E50E94DB1BCF910C94761C843859F4E1
:102460000E94EF1082FD9DC087E40E94991B0E948C
:10247000761C87E4EECF8CEF8C0F813A48F48C2FDA
:102480000E94E42181118DC08C2F0E94991BE3CF03
:1024900080E28C0F883048F4C77081E001C0880F5B
:1024A000CA95EAF70E94221CD6CF8BE58C0F8330A9
:1024B00078F4C53A29F0C63A31F083E890E005C0D7
:1024C00081E890E002C082E890E0CF910C94111175
:1024D00088E58C0F833108F064C0C83A39F1C93AF5
:1024E00041F1CA3A49F1CB3A51F1CC3A59F1CD3ADE
:1024F00061F1C03B69F1CE3A71F1CF3A79F1C13B5C
:1025000081F1C23B89F1C33B91F1C43B99F1C53BD9
:10251000A1F1C63BA9F1C73BB1F1C83BB9F1C93B39
:10252000C1F1CA3BC9F180E090E038C082EE90E092
:1025300035C089EE90E032C08AEE90E02FC085EB86
:1025400090E02CC086EB90E029C087EB90E026C09D
:102550008CEC90E023C08DEC90E020C083E891E00B
:102560001DC08AE891E01AC082E991E017C084E9B1
:1025700091E014C081E292E011C083E292E00EC0CB
:1025800084E292E00BC085E292E008C086E292E02D
:1025900005C087E292E002C08AE292E0CF910C94FB
:1025A0002711CF910895882309F44BC0823859F43C
:1025B0000E94EF1081FF45C089E30E94991B0E9491
:1025C000761C89E30CC0833871F40E94EF1080FF01
:1025D00038C083E50E94991B0E94761C83E50E9407
:1025E000DB1B0C94761C843859F40E94EF1082FF98
:1025F00028C087E40E94991B0E94761C87E4EFCFD5
:102600009CEF980F913A58F390E2980F983050F45D
:10261000877091E001C0990F8A95EAF7892F0E948F
:10262000281CDFCF9BE5980F933020F480E090E0EA
:102630000C941111885A833120F480E090E00C94BE
:1026400027110895882321F00E94221C0C94761CE7
:102650000895882321F00E94281C0C94761C08956C
:102660008F929F92AF92BF92DF92EF92FF920F9361
:102670001F93CF93DF937C01D62FC72FFC010281DC
:10268000158112951F700E94351B882319F082E076
:102690000E94771B01110E943F1C0E94921B8823FD
:1026A00079F0002369F080E28D0F883048F082E0F5
:1026B0000E94771B0E94921B91E0D82ED92601C060
:1026C000D12CEC2FE295EF70F0E0E05AFF4F0C9424
:1026D00018248C2F807FCF70882311F0C295C07F83
:1026E000002389F0CC2309F4C4C180E28D0F883027
:1026F00020F48C2F0E94221C03C08C2F0E94321CBD
:102700000E94761CB6C18D2F0E94D312CC2309F4EF
:10271000CAC1D05E8C2FD83018F40E94281C02C089
:102720000E94381C0E94761CBEC18C2F807FCF7007
:10273000803211F0C295C07FDD2319F0D13029F12C
:102740002DC0002381F0112369F1113021F48C2F69
:102750000E94521CA8C1123029F50E945B1C8C2FCC
:102760000E94021B1FC0112369F0113041F40E9426
:102770001F1C8C2309F497C10E94051B03C0123053
:1027800009F491C10E945B1C11C0002321F012309A
:1027900008F089C107C0111186C108C0002321F0CB
:1027A000111167C18C2FF1C011116AC18C2FF3C0B8
:1027B0008C2F86958695837090E0009719F001978D
:1027C00061F071C1002321F08D2F9C2F937002C006
:1027D00080E090E00E94111166C1002321F08D2F4E
:1027E0009C2F937002C080E090E00E9427115BC193
:1027F0008D2F002319F00E94A21E02C00E940A1F02
:102800000E948F1F50C18C2F837009F050C001119E
:102810004AC18D2F829586958770880F880F9D2FCE
:102820009F70892E912CA12CB12C082E04C0880CED
:10283000991CAA1CBB1C0A94D2F7D4FF14C00FE049
:1028400010E020E030E0B901A80104C0440F551F9A
:10285000661F771F8A95D2F7CB01BA0160957095F4
:102860008095909503C060E070E0CB01C695C69559
:10287000C370D0E0C230D10561F0C330D10581F022
:10288000682979298A299B29219771F00E949E192C
:102890000AC1682979298A299B290E94BA1903C18A
:1028A0000E949E19C501B4010E948219FCC0002338
:1028B00019F08C2F817001C08695882309F4F3C02C
:1028C0008D2F829586958770880F880F9D2F9F701A
:1028D000892E912CA12CB12C082E04C0880C991C97
:1028E000AA1CBB1C0A94D2F7D4FF14C00FE010E05E
:1028F00020E030E0B901A80104C0440F551F661F55
:10290000771F8A95D2F7CB01BA01609570958095B3
:10291000909503C060E070E0CB01C695C695C3708A
:102920004C2F50E04230510569F04330510589F099
:10293000682979298A299B294130510571F00E9423
:10294000781AB1C0682979298A299B290E94941A8A
:10295000AAC00E94781AC501B4010E945C1AA3C0E3
:102960008D2F90E0FC01E05EF109E531F10508F002
:102970007BC0E059FF4F0C941824DF708C2F8F71AF
:10298000002331F00E94F5198D2F0E9422138BC075
:102990000E94161A8D2F0E94291385C0002339F03A
:1029A000111181C08C2F8F710E943B1A7CC0123094
:1029B00008F079C0F7CF002339F08C2F8F710E9477
:1029C000F51971C00023C9F38C2F8F710E94161A5C
:1029D0006AC0002329F08C2F8F710E94E01963C018
:1029E0000E94D61960C00023B9F00E94FF1A0E940D
:1029F000281C0E94311B843029F40E94701B8C2FEC
:102A00008F7162C0123008F06CC0CF718C2F0E94A1
:102A1000F51963E08C2F0DC00E94FF1A0E94221C42
:102A20001230A0F00E94701B0E94051B64E08C2FE6
:102A30008F71DF91CF911F910F91FF90EF90DF90F9
:102A4000BF90AF909F908F900C94601B81E0DF91BE
:102A5000CF911F910F91FF90EF90DF90BF90AF90BB
:102A60009F908F900C94771B002339F0112309F469
:102A7000A4CF8D2F0E940B1216C0112309F4A4CFEE
:102A80008D2F0E94D3120FC04C2F4F706D2FC70196
:102A90000E9446050E94FA1806C04C2F4F706D2FF9
:102AA000C7010E945B09DD20E1F00E94311B80FD1F
:102AB00018C0F70112820E942B1B0E94F519C70152
:102AC0000E947D150E942B1BDF91CF911F910F91CA
:102AD000FF90EF90DF90BF90AF909F908F900C94FD
:102AE000161ADF91CF911F910F91FF90EF90DF9019
:102AF000BF90AF909F908F9008950F931F93CF93A7
:102B0000DF93EC01888199812B813C81232BB9F0E3
:102B10009F3F11F48F3F99F0CE010E94EC0588236E
:102B200071F0688179818A810E94FB1A8C010E9470
:102B3000B01A0E947719B801CE010E943013DF91BC
:102B4000CF911F910F9108950E943F1C0E944F1C2E
:102B50000E94111C0E94761C0E9440200E948F1F20
:102B600080E090E00E94111180E090E00C94271129
:102B70000E942F1C0C94A4150E94F01A292F229554
:102B80002F7030E02C3031054CF42A3031056CF4D4
:102B90002250310922303105A8F407C02C3031050C
:102BA00069F02F30310551F00DC0803F69F018F405
:102BB000803E40F409C0843F29F406C093FB882777
:102BC00080F9089580E0089581E00895CF93DF9320
:102BD00000D000D01F92CDB7DEB70F900F900F90AE
:102BE0000F900F90DF91CF910895CF93DF9300D096
:102BF00000D000D0CDB7DEB726960FB6F894DEBF72
:102C00000FBECDBFDF91CF9108951F93CF93DF9378
:102C1000C091870116E080918801C81799F0D0E033
:102C20001C9FF0011D9FF00D1124E757FE4F4081BE
:102C3000518162817381848195810E94F51521966D
:102C4000C770E9CFDF91CF911F9108954091B901ED
:102C50005091BA016091BB017091BC018091BD019E
:102C60009091BE010C94F5158091BE0182958F70F4
:102C700009F054C08091BB01882309F44FC08091B2
:102C80008701A09188016091B9017091BA014091CA
:102C9000BC015091BD01B6E08A1709F43FC090E035
:102CA00041155105C1F17F3F11F46F3FA1F1B89F6C
:102CB000F001B99FF00D1124E757FE4F21817213E7
:102CC0002AC02081621327C02281211124C02381C0
:102CD00034812417350710F421503109241B350B9A
:102CE000283C3105C0F42091BE012F702061209353
:102CF000BE0126E0289FF001299FF00D1124E25724
:102D0000FE4F80818F708061808389EB91E00E940B
:102D10007D150C94051601968770BECF0895CF924D
:102D2000DF92EF92FF920F931F93CF93DF93CDB774
:102D3000DEB762970FB6F894DEBF0FBECDBF8C0131
:102D400085E0F801DE011D9601900D928A95E1F76C
:102D5000D8014C9111965C91119712966C91129733
:102D60001396CD90DC9014973091B9017091BA010F
:102D70008091BC019091BD01009709F46BC17F3F28
:102D800019F43F3F09F466C1E090BB01EE2009F45D
:102D9000C0C02091BE01C816D90628F0F601E81B74
:102DA000F90BCF0104C0809590958C0D9D1DFF24DB
:102DB000F394883C910578F0F12C207F09F0C6C08F
:102DC0007C2DD98AC88A89890E94E61589EB91E011
:102DD0000E947D15B1C0822F807F09F046C0751317
:102DE00014C0341312C0611110C02F7020612093E1
:102DF000BE010E94261689EB91E00E947D1580910C
:102E0000BE01D80115968C932EC0CD2819F15F3FD5
:102E100011F44F3FF9F0F62E61111CC0809187012B
:102E20002091880136E0821709F45AC090E0389F5B
:102E3000F001399FF00D1124E757FE4F71815713B0
:102E400006C07081471303C07281711103C00196DF
:102E50008770E9CFF62E662309F418C18091BE0170
:102E600081608093BE01F12C11C1751308C0341329
:102E700006C0611104C08091BE01D801C3C04D8756
:102E80005E878D859E856A8B0E94BC156A89882322
:102E9000E1F16623D1F12091BE01822F82958F70DE
:102EA00090E0029774F08091B9019091BA019887EF
:102EB0008F831986DB86CA862C87CE0107960E94EF
:102EC0007D1586E0F801A9EBB1E001900D928A959D
:102ED000E1F70E9434160E942616FF24F394D6C010
:102EE0004D875E878D859E850E94F01A292F229539
:102EF0002F7030E0223031050CF0BCC09F7009F01B
:102F0000B6C0805E883008F4C1C0C8010E947D153B
:102F1000E4CFC816D90608F453C0F601E81BF90B34
:102F2000CF01883C910508F450C0F12C7C2DD98A42
:102F3000C88A89890E94E615E9EBF1E086E0DF01A5
:102F40001D928A95E9F70E942616A0C0751314C039
:102F5000341312C0611110C08091BE01F801858345
:102F6000C8010E947D1586E0E9EBF1E0DF011D92CA
:102F70008A95E9F7FE2C8AC04D875E878D859E85F0
:102F80006A8B0E94BC156A89882309F4BECF662328
:102F900009F4BBCF2091BE01822F82958F7090E003
:102FA00002970CF48ECF8091B9019091BA019A8367
:102FB00089831B82DD82CC822E83CE0101967FCF56
:102FC000809590958C0D9D1DACCFF62E662309F44F
:102FD0009CCF75132EC034132CC02091BE0120FD50
:102FE0001FC0822F82958F70D9F0D80115962C932F
:102FF00015978F3049F08F5F982F9295907F822F91
:103000008F70892B15968C93C8010E947D1586E0E0
:10301000F801A9EBB1E001900D928A95E1F793CF09
:1030200086E0F801A9EBB1E001900D928A95E1F7F5
:103030002DC04D875E878D859E850E94BC158111B0
:1030400040CF8091BE0181608093BE01C8010E9483
:103050007D151CC0662309F458CF4D875E878D858A
:103060009E850E94BC15882309F44FCF2ACF811179
:1030700048CF0CC0243031050CF047CF9F7009F4C5
:1030800040CFF8019581907F09F03BCF8F2D62965C
:103090000FB6F894DEBF0FBECDBFDF91CF911F9169
:1030A0000F91FF90EF90DF90CF9008951F93CF93F3
:1030B000DF93CDB7DEB72C970FB6F894DEBF0FBE07
:1030C000CDBF4F83588769877A878B879C87CE01CE
:1030D00007960E948F16882369F08F8198852A852C
:1030E0003B85232BF1F19F3F09F063C08F3F09F02F
:1030F00060C037C086E0FE013796DE011196019070
:103100000D928A95E1F76F817885EA85FB85309786
:1031100041F17F3F11F46F3F21F12091880130E0B0
:10312000C9010196877099274091870150E0841763
:10313000950709F447C069837A83FD83EC8396E0A1
:10314000929FD001939FB00D1124A757BE4FFE014F
:10315000319601900D929A95E1F7809388010E9433
:10316000051616E080918701909188018917C1F1B9
:10317000189FC001112487579E4F0E948F168823E5
:1031800079F1E09187011E9FF0011124E757FE4F6E
:103190004081518162817381848195810E94F515FE
:1031A0008091870190E0019687709927809387012D
:1031B000D9CF4F81588569857A858B859C850E94FA
:1031C000F515CFCF0E94B815109288011092870193
:1031D000E9EBF1E086E0DF011D928A95E9F7C1CFC6
:1031E0002C960FB6F894DEBF0FBECDBFDF91CF9106
:1031F0001F910895EF92FF920F931F93CF93DF9348
:103200008C01009709F46CC0F12CEE24E394E801E2
:103210002196F8018491843740F4843008F051C03D
:10322000813081F0823019F15BC0853709F444C0E8
:10323000A8F19CE7980F903708F052C08F770E9452
:10324000D31241C00E5F1F4FFE01C49180E28C0F6C
:10325000883048F4C7708E2D01C0880FCA95EAF7F0
:103260000E94421C14C08C2F0E940B122DC00E5FB6
:103270001F4FFE01C49180E28C0F883058F4C77054
:103280008E2D01C0880FCA95EAF70E94481C0E9443
:10329000761C1AC08C2F0E94D31216C00E5F1F4FCF
:1032A000FE01C491CC2381F08FE99FE00197F1F7F3
:1032B00000C00000C150F6CF0E5F1F4FFE01F4901A
:1032C00003C00E940B128E018F2D882309F49FCF1B
:1032D000EFE9FFE03197F1F700C000008150F5CF32
:1032E000DF91CF911F910F91FF90EF900895089576
:1032F0006093C3017093C4018093C5019093C6018C
:103300000C94A4150F931F930091C3011091C40155
:103310002091C5013091C601DC01CB01802B912B9E
:10332000A22BB32B8093C3019093C401A093C5013A
:10333000B093C6011F910F910C94A4150F931F9386
:103340000091C3011091C4012091C5013091C601C3
:10335000DC01CB0180239123A223B3238093C301FB
:103360009093C401A093C501B093C6011F910F9122
:103370000C94A4150F931F930091C3011091C401E5
:103380002091C5013091C601DC01CB018027912736
:10339000A227B3278093C3019093C401A093C501D2
:1033A000B093C6011F910F910C94A4151092BF0108
:1033B0001092C0011092C1011092C2010C94A41588
:1033C00041E050E060E070E004C0440F551F661F0C
:1033D000771F8A95D2F74093BF015093C001609345
:1033E000C1017093C2010C94A41541E050E060E06B
:1033F00070E004C0440F551F661F771F8A95D2F7EF
:103400008091BF019091C001A091C101B091C20112
:10341000482B592B6A2B7B2B4093BF015093C00143
:103420006093C1017093C2010C94A41541E050E077
:1034300060E070E004C0440F551F661F771F8A9537
:10344000D2F740955095609570958091BF0190910D
:10345000C001A091C101B091C201482359236A2340
:103460007B234093BF015093C0016093C1017093CF
:10347000C2010C94A41541E050E060E070E004C08B
:10348000440F551F661F771F8A95D2F78091BF01A1
:103490009091C001A091C101B091C2014827592764
:1034A0006A277B274093BF015093C0016093C101FD
:1034B0007093C2010C94A4150F931F930091BF0148
:1034C0001091C0012091C1013091C201DC01CB01FA
:1034D000802B912BA22BB32B8093BF019093C00123
:1034E000A093C101B093C2011F910F910C94A41538
:1034F0000F931F930091BF011091C0012091C10152
:103500003091C201DC01CB0180239123A223B3239C
:103510008093BF019093C001A093C101B093C201F9
:103520001F910F910C94A4150F931F930091BF014D
:103530001091C0012091C1013091C201DC01CB0189
:1035400080279127A227B3278093BF019093C001C2
:10355000A093C101B093C2011F910F910C94A415C7
:103560000895CF92DF92EF92FF920F931F93CF9324
:10357000DF938C01C090C301D090C401E090C501DD
:10358000F090C6018091BF019091C001A091C1014E
:10359000B091C201C82AD92AEA2AFB2ACFE1D0E099
:1035A000D701C6010C2E04C0B695A79597958795AF
:1035B0000A94D2F780FF06C0B8018C2F0E94DA0768
:1035C000019721F4219760F780E001C08C2FDF91F3
:1035D000CF911F910F91FF90EF90DF90CF900895C2
:1035E000CF93DF93EC010E94B11ABE010E94DA076B
:1035F000DF91CF910895CB010E94F01A0895809138
:10360000CC0108958093CC0108951092CC010895C7
:103610000E944F1D2091CA013091CB018217930760
:1036200050F00E944F1D2091CA013091CB01821BA6
:10363000930B9C010AC00E944F1D2091CA0130913A
:10364000CB0120953095280F391F81E0283B3B4066
:1036500008F480E008958091C90185958595859548
:1036600008958091C901877008950E944F1D20918F
:10367000C7013091C80182179307A8F00E944F1D1F
:103680002091C7013091C801821B930B883B9B405E
:1036900010F480E013C08091C90182FB882780F973
:1036A00091E089270BC00E944F1D2091C7013091E6
:1036B000C80120953095820F931FE8CF817008953F
:1036C00098E0899F90011124262B2093C9010E9424
:1036D000F5190E944F1D9093C8018093C70108956A
:1036E0001092C9011092C8011092C701089520914B
:1036F000C901809582238093C901982F977089F41E
:1037000030E0482F552747FD50952417350749F0DD
:103710008595859585950E94161A1092C80110927C
:10372000C70108959091C901977081E009F480E084
:10373000089590910C01992321F090910D01911120
:1037400009C020910E0130910F01F90132969FEFCF
:1037500040E01FC0982F9695969596959F3050F50E
:10376000E0910E01F0910F01E90FF11D877021E04A
:1037700030E0A90102C0440F551F8A95E2F7CA0143
:103780009181892B818308959F3F39F04F5F4E309F
:1037900041F051915813F8CF0DC05111F7CF942F2C
:1037A000F5CF9F3F39F0F901E90FF11D97FDFA952B
:1037B00082830895089590910C01992321F09091AE
:1037C0000D01911109C020910E0130910F01F901F5
:1037D0003296205F3F4F1FC0982F969596959695ED
:1037E0009F30F0F4E0910E01F0910F01E90FF11D0F
:1037F000877021E030E0A90102C0440F551F8A956F
:10380000E2F7CA01809591818923818308953196D9
:10381000E217F30729F090819813F9CF1082F7CFC0
:10382000089581E090E0E0910E01F0910F01E80F22
:10383000F91F1082019680319105A9F708958091B2
:10384000E00108959091E001892B8093E0010895B3
:1038500080959091E00189238093E0010895109272
:10386000E00108959091DF01892B8093DF01089595
:1038700080959091DF0189238093DF010895109254
:10388000DF0108959091DE01892B8093DE01089578
:1038900080959091DE0189238093DE010895109236
:1038A000DE0108958093CD010E944F1D9093CB01BE
:1038B0008093CA0108951092CD011092CB0110920D
:1038C000CA0108958091CD01089580910E019091D3
:1038D0000F01FC0131969C01205F3F4F80E09191E8
:1038E00091118F5FE217F307D1F70895E0910E0170
:1038F000F0910F018091E0018083E0910E01F09141
:103900000F0190818091DF01892B8083E0910E016E
:10391000F0910F0190818091DE01892B808380914D
:10392000CD01882399F00E94081B81110E945B1C25
:10393000E0910E01F0910F0190818091CD01892BD2
:1039400080830E94651C81110E945B1C80910E0186
:1039500090910F010C94FB1020E0009739F0AC011E
:1039600041505109842395232F5FF7CF822F08956B
:10397000CF92DF92EF92FF926C01EE24FF24C114EC
:10398000D104E104F10421F0C701B60120E101C036
:1039900020E0C72ED82EE92EFF24C114D104E10463
:1039A000F10419F0285FC701B6016B017C0154E0F6
:1039B000F694E794D794C7945A95D1F7C114D104DB
:1039C000E104F10419F02C5FC701B6016B017C0121
:1039D00042E0F694E794D794C7944A95D1F7C1147E
:1039E000D104E104F10419F02E5FC701B601DC0136
:1039F000CB01B695A79597958795892B8A2B8B2B0D
:103A000009F02F5F822FFF90EF90DF90CF90089505
:103A10008091FA01843021F11092E20120E488E1E2
:103A200090E00FB6F894A895809360000FBE2093A5
:103A3000600080E00E94EC0983B7817F846083BFCF
:103A400083B7816083BF7894889583B78E7F83BF67
:103A500088E10FB6F89480936000109260000FBE6A
:103A6000089508950E9469030E947C030E94311DFD
:103A70000E94710491E0811101C090E0892F0895A6
:103A80000E94B8150E94EF100C94EC0982E084BDEE
:103A900093E095BD9AEF97BD80936E0008952FB780
:103AA000F8948091E3019091E401A091E501B09137
:103AB000E6012FBF0895CF92DF92EF92FF920F930E
:103AC0001F932FB7F8944091E3015091E401609166
:103AD000E5017091E6012FBF6A017B01EE24FF240E
:103AE0008C0120E030E0C016D106E206F30610F4A7
:103AF000415051099A01281B390BC9011F910F919F
:103B0000FF90EF90DF90CF9008951F920F920FB625
:103B10000F9211248F939F93AF93BF938091E301F2
:103B20009091E401A091E501B091E6010196A11DFB
:103B3000B11D8093E3019093E401A093E501B0935C
:103B4000E601BF91AF919F918F910F900FBE0F90A3
:103B50001F9018950E94EC0DF8942FEF87EA91E6DC
:103B6000215080409040E1F700C0000087E090EBDA
:103B7000DC018093030290930402A0930502B093AA
:103B800006029CE088E10FB6F894A8958093600047
:103B90000FBE90936000FFCF0E94041E811102C0EF
:103BA0000E94EA1D0E940F1E8093E1010E94171ED1
:103BB00090E09093F5018093F40187FB882780F9CA
:103BC00080930D010E94131E682F70E080E090E04A
:103BD0000C9478196DEE7EEF80E090E00E94522404
:103BE00060E082E090E00E94402460E083E090E0AA
:103BF0000E94402460E084E090E00E94402460E065
:103C000085E090E00C94402480E090E00E943A240B
:103C100021E08D3E9E4F09F020E0822F089582E042
:103C200090E00C94322483E090E00C94322484E001
:103C300090E00C943224682F84E090E00C944024AF
:103C40008091E90180FF0BC06091130185E0689FBE
:103C5000B001112475956795759567952BC081FF07
:103C600009C06091130185E0689FB001112475952A
:103C7000679520C082FF07C06091130185E0689FAF
:103C8000B001112417C09091EA019923D1F06091FD
:103C90001201961788F72091130185E0289F900163
:103CA0001124929FA001939F500D112470E0CA012E
:103CB0000E9404246038710540F46115710539F0E3
:103CC00002C065E070E0862F08958FE7089581E0D7
:103CD00008958091E90180FF08C06091110170E0B2
:103CE000759567957595679521C081FF06C06091B0
:103CF000110170E07595679519C082FF04C060914D
:103D0000110170E010C09091EA019923C1F0609117
:103D100010019617A0F780911101899FC00111240D
:103D200070E00E9404246038710528F46115710563
:103D300021F0862F08958FE7089581E0089561E0CE
:103D400070E0F4CF803F21F40E94201E819504C0D2
:103D5000813F29F40E94201E8093ED010895823F47
:103D600021F40E94201E819504C0833F29F40E9403
:103D7000201E8093EC010895893F19F40E94691E6A
:103D800005C08A3F31F40E94691E81958093EE013F
:103D900008958B3F21F40E94691E819504C08C3FD9
:103DA00029F40E94691E8093EF010895843F21F455
:103DB0008091EB01816017C0853F21F48091EB0178
:103DC000826011C0863F21F48091EB0184600BC0BA
:103DD000873F21F48091EB01886005C0883F31F472
:103DE0008091EB0180618093EB0108958D3F21F478
:103DF0008091E90181600BC08E3F21F48091E9013F
:103E0000826005C08F3F29F48091E901846080932E
:103E1000E9010895803F39F48091ED0187FF6CC07E
:103E20001092ED0169C0813F29F48091ED011816CF
:103E3000BCF362C09091EC01823F29F497FF5CC013
:103E40001092EC0159C0833F19F41916CCF354C0F9
:103E5000893F41F48091EE0118160CF04DC010928C
:103E6000EE014AC08A3F29F48091EE0187FF44C0E9
:103E7000F6CF8B3F39F48091EF0187FF3DC0109260
:103E8000EF013AC08C3F29F48091EF011816BCF382
:103E900033C0843F21F48091EB018E7F17C0853FB2
:103EA00021F48091EB018D7F11C0863F21F4809138
:103EB000EB018B7F0BC0873F21F48091EB01877F63
:103EC00005C0883F31F48091EB018F7E8093EB0138
:103ED00013C08D3F21F48091E9018E7F0BC08E3F8E
:103EE00021F48091E9018D7F05C08F3F29F48091F5
:103EF000E9018B7F8093E9018091EC0181110EC073
:103F00008091ED0181110AC08091EE01811106C0FE
:103F10008091EF01811102C01092EA0108958BEEA9
:103F200091E00E9406110E944F1D9093E80180933A
:103F3000E70108951F93CF93DF938091E70190915C
:103F4000E8010E945B1DAC019091EA01992321F0E8
:103F50002091140130E006C0209115018AE0289FCD
:103F6000900111244217530708F486C08091EC0198
:103F7000C091ED01D091EE011091EF01811107C0C8
:103F8000C11176C0D11174C0111172C075C09F3FAC
:103F900019F09F5F9093EA01181624F40E94201EE6
:103FA0008093EC018091EC0187FF05C00E94201EE8
:103FB00081958093EC011C1624F40E94201E8093AE
:103FC000ED018091ED0187FF05C00E94201E8195C3
:103FD0008093ED016091EC01662339F1C091ED0110
:103FE000CC2319F1772767FD7095872F972F0E94B3
:103FF000152323E333E343E35FE30E9479230E9425
:10400000E2226093EC016C2F772767FD7095872F74
:10401000972F0E94152323E333E343E35FE30E94DA
:1040200079230E94E2226093ED011D1624F40E9480
:10403000691E8093EE018091EE0187FF05C00E940A
:10404000691E81958093EE01111624F40E94691E69
:104050008093EF018091EF0187FF05C00E94691EE8
:1040600081958093EF01DF91CF911F910C948F1F69
:104070009F3F09F08ECF96CFDF91CF911F9108958A
:10408000EBEEF1E085E0DF011D928A95E9F71092F1
:10409000EA011092E9010895833081F128F481301A
:1040A00059F08230D1F00895853009F449C0B8F153
:1040B000863009F456C0089580911501262F30E00E
:1040C000280F311D2F3F310524F4680F609315012F
:1040D00008958FEF80931501089580911401262F84
:1040E00030E0280F311D2F3F310524F4680F609315
:1040F000140108958FEF80931401089580911301A6
:10410000262F30E0280F311D2F3F310524F4680F92
:104110006093130108958FEF8093130108958091A8
:104120001201262F30E0280F311D2F3F310524F4D6
:10413000680F6093120108958FEF80931201089524
:1041400080911101262F30E0280F311D2F3F3105BE
:1041500024F4680F6093110108958FEF809311018B
:10416000089580911001262F30E0280F311D2F3F38
:10417000310524F4680F6093100108958FEF809348
:1041800010010895833011F128F4813049F0823014
:1041900091F00895853081F120F18630C1F10895C4
:1041A00080911501681720F4861B809315010895EE
:1041B00010921501089580911401681720F4861B50
:1041C00080931401089510921401089580911301B1
:1041D000681720F4861B8093130108951092130131
:1041E000089580911201681720F4861B80931201B4
:1041F000089510921201089580911101681720F41A
:10420000861B8093110108951092110108958091E9
:104210001001681720F4861B8093100108951092F6
:10422000100108950F931F938D3109F471C008F0A8
:1042300045C0803109F485C008F5873009F46FC0A6
:1042400068F4863009F0ADC08091E101817F8E7FF6
:104250008093E10181E08093F101A4C08B3009F4E7
:104260009EC08E3009F09DC08091E10182FB222723
:1042700020F991E0922790FB82F96CC0863109F415
:104280008EC060F4813109F08CC00E94B815909105
:104290000D0181E0892780930D0181C0893109F4E6
:1042A0007EC08B3109F07DC08091E10181FB222726
:1042B00020F991E0922790FB81F94CC0853309F4F5
:1042C00066C048F4873209F462C008F44FC08932EE
:1042D00009F45DC066C0833438F48A3308F044C002
:1042E000883309F45CC05DC0833409F450C088345D
:1042F00009F057C00E94B8150FEF13ED20E30150ED
:1043000010402040E1F700C000000E94AA1D47C0F5
:104310000E949C220E94EF100E94EC0940C09091E4
:10432000E101892F8095817080FB90F929F09660DA
:1043300098609093E10136C0997F977F9093E10157
:104340002EC08091E10183FB222720F991E0922782
:1043500090FB83F98093E101992309F18091E101B8
:1043600081608093E1011BC0895301C08D5141E000
:1043700050E060E070E08A019B0104C0000F111F53
:10438000221F331F8A95D2F7C901B80104C061E02A
:1043900070E080E090E00E9478190E94B81581E0FA
:1043A00001C080E01F910F91089580E0089580E0A2
:1043B00008958E518A3030F4E82FF0E0E65DFE4F2C
:1043C0008081089580E00895CF93C82F8091F101F6
:1043D000813079F018F08230E9F186C0E0910E0169
:1043E000F0910F018081813169F0823209F07EC045
:1043F00009C0E0910E01F0910F018081813111F02F
:10440000823261F48C2F0E94D521811104C08C2F3F
:104410000E9412211DC081E090E01AC08C2F0E94E2
:10442000D721811114C0C43179F048F4CB3079F030
:10443000C03109F05FC082E08093F10108C0C93249
:1044400019F0C83321F056C01092F10153C081E039
:10445000817052C0C93281F110F5C43169F1A8F4FC
:10446000C73009F045C08AE08093150194E190932C
:10447000140193E0909313018093120188E08093DC
:10448000110188E28093100133C082EE8C0F8630D8
:1044900078F58C2F0E94D9218093F00129C0CE3469
:1044A000E9F020F4CB3421F56AE013C0C13579F08E
:1044B000C235F1F461E00DC08091F001882319F05C
:1044C0001092F00115C081E08093F10115C061E008
:1044D00006C08091F0010E944C200AC06AE08091E1
:1044E000F0010E94C22004C01092F10180E004C0DB
:1044F00081E002C080E0ACCFCF910895E1E8F0E028
:104500008081886080838081816080838FB7F89408
:1045100093E09093890090ED909388008FBF089569
:10452000EFE6F0E08081826080830895EFE6F0E0BE
:1045300080818D7F80830895EFE6F0E0908182E0B6
:104540008927808308951F920F920FB60F9211242E
:104550002F933F934F935F936F937F938F939F938B
:10456000AF93BF93EF93FF938091F2019091F3018A
:1045700001969093F3018093F201811103C082E0D0
:104580000E94EC09E091F301E695E695F0E0E75131
:10459000FB4FE4918091F2018E1303C080E00E94F2
:1045A000EC09FF91EF91BF91AF919F918F917F9116
:1045B0006F915F914F913F912F910F900FBE0F9090
:1045C0001F90189504D06894B1118DC0089570D0D3
:1045D00088F09F5790F0B92F9927B751A0F0D1F0EC
:1045E000660F771F881F991F1AF0BA95C9F712C076
:1045F000B13081F077D0B1E0089574C0672F782F83
:104600008827B85F39F0B93FCCF3869577956795E1
:10461000B395D9F73EF490958095709561957F4F4D
:104620008F4F9F4F0895E89409C097FB3EF49095F3
:104630008095709561957F4F8F4F9F4F9923A9F07B
:10464000F92F96E9BB279395F6958795779567950A
:10465000B795F111F8CFFAF4BB0F11F460FF1BC04E
:104660006F5F7F4F8F4F9F4F16C0882311F096E9E1
:1046700011C0772321F09EE8872F762F05C066238F
:1046800071F096E8862F70E060E02AF09A95660F48
:10469000771F881FDAF7880F9695879597F9089501
:1046A00057FD9058440F551F59F05F3F71F04795E3
:1046B000880F97FB991F61F09F3F79F087950895C8
:1046C000121613061406551FF2CF4695F1DF08C0E7
:1046D000161617061806991FF1CF86957105610504
:1046E00008940895E894BB2766277727CB0197F9AC
:1046F00008950BD078C069D028F06ED018F09523BB
:1047000009F05AC05FC01124EECFCADFA0F3959F15
:10471000D1F3950F50E0551F629FF001729FBB27A8
:10472000F00DB11D639FAA27F00DB11DAA1F649F54
:104730006627B00DA11D661F829F2227B00DA11D07
:10474000621F739FB00DA11D621F839FA00D611D8D
:10475000221F749F3327A00D611D231F849F600DAE
:10476000211D822F762F6A2F11249F5750408AF0E7
:10477000E1F088234AF0EE0FFF1FBB1F661F771F73
:10478000881F91505040A9F79E3F510570F014C00A
:10479000AACF5F3FECF3983EDCF38695779567955B
:1047A000B795F795E7959F5FC1F7FE2B880F911D91
:1047B0009695879597F9089597F99F6780E870E037
:1047C00060E008959FEF80EC089500240A94161687
:1047D000170618060906089500240A9412161306EF
:1047E000140605060895092E0394000C11F488237D
:1047F00052F0BB0F40F4BF2B11F460FF04C06F5F99
:104800007F4F8F4F9F4F089597FB072E16F400940C
:1048100007D077FD09D00E941E2407FC05D03EF486
:10482000909581959F4F0895709561957F4F08955C
:10483000EE0FFF1F0590F491E02D0994AA1BBB1BFE
:1048400051E107C0AA1FBB1FA617B70710F0A61B90
:10485000B70B881F991F5A95A9F780959095BC01B1
:10486000CD010895F999FECF92BD81BDF89A99279F
:1048700080B50895A8E1B0E042E050E00C945A24DD
:10488000262FF999FECF92BD81BDF89A019700B409
:10489000021639F01FBA20BD0FB6F894FA9AF99AA9
:1048A0000FBE08950196272F0E9441240C944024A6
:1048B000DC01CB01FC01F999FECF06C0F2BDE1BDE0
:1048C000F89A319600B40D9241505040B8F70895CF
:0448D000F894FFCF8A
:1048D4000220EE097C0A590A250AF1090101CE01D8
:1048E40028080A03140A404D3639A9045C04260436
:1048F400ED0380039903B203CB030102030405060D
:044904000708090097
:00000001FF
